:020000040000FA
:10000000831600308600831200308600FF308600A1
:100010002D210F202D21000040202D210B287220A2
:10002000003086007E200614A0308F0091208617B5
:10003000792018212D2172208613861400308F001C
:1000400091208617792018212D21722086130615FC
:10005000FF308F0091208617792018212D217220E2
:1000600086138615F0308F0091208617792018218D
:100070002D2172208613851588202D2185110034AD
:100080007220003086007E200614A0308F00912060
:100090008617792018212D217220861386140030AE
:1000A0008F0091208617792018212D217220861328
:1000B0000615FF308F0091208617792018212D21F9
:1000C0008613861572207E200515A1308F009120A1
:1000D000051179201821DB207220851588202D211B
:1000E00085110034831600308500831200308500AE
:1000F0000034831601308500831200340514851006
:100100002D2185142D2105102D2185102D21003440
:1001100005102D2185142D2105142D2185102D214B
:10012000003485102D218F1B05148F1F05102D21E4
:1001300085142D2185102D210F1B05140F1F05106F
:100140002D2185142D2185102D218F1A05148F1E28
:1001500005102D2185142D2185102D210F1A051430
:100160000F1E05102D2185142D2185102D218F198D
:1001700005148F1D05102D2185142D2185102D218D
:100180000F1905140F1D05102D2185142D21851023
:100190002D218F1805148F1C05102D2185142D215C
:1001A00085102D210F1805140F1C05102D21851405
:1001B0002D21851000342D21851405188617051C66
:1001C000861385102D21851405180617051C0613A6
:1001D00085102D21851405188616051C861285109C
:1001E0002D21851405180616051C061285102D21D3
:1001F000851405188615051C861185102D2185147A
:1002000005180615051C061185102D2185140518E5
:100210008614051C861085102D21851405180614DA
:10022000051C061085102D2185142D218510003404
:100230000430900085142D21051C2129900B1C29C8
:10024000232185100034003086002D21FF308600E8
:100250002D21003086002D21003402308E00F03038
:100260008C00F0308D008D0B33298C0B31298E0BD7
:040270002F290034FE
:02400E00F93F78
:00000001FF
